:020000020000FC
:040000000DC01AC154
:0200120052C0DA
:10001A0074C000EF0ABB08E00BBB03E007BB04E0B7
:10002A0008BB0FED0DBF00E40BBF01E205BF00E8FE
:10003A0008B90AE000B907E001B902E000BF04E02C
:10004A0003BF0DE406BF02E009BF34E161E021E02D
:10005A00CC27DD27EE27FF27772788279927AA2786
:10006A00BB27EE24FF24002700936200009363005D
:10007A0000936600009367000FEF009360000093FF
:10008A0064000093610000936500002700936800F4
:10009A000093690000936A00F8940BE006B978941B
:1000AA008895FACF0BE806B9789488950895E030D8
:1000BA00D9F42A9531F42CEDEC0101E0070F046024
:1000CA0008BB283719F4ED0104E008BB253160F4B8
:1000DA00022F0A950695C9E0C01BDC2F04E008BB75
:1000EA0002E0071B046008BBF03021F0FA9511F416
:1000FA00EE2725E1A5D0D6DF189504B115B1E00E9B
:10010A00F11E6A9551F467E209D03A9509F432E092
:10011A00032F01700395006407B91895F694E794C4
:10012A00F694E794F694E794F694E794A70130FFDF
:10013A0042C03330B0F41091610000916000E016C3
:10014A00F10620F4F0926100E092600010916300E1
:10015A00009162000E151F0520F4F0926300E092F0
:10016A006200FF24EE247727463D05E05007F0F4AD
:10017A00443F01E0500718F04F5E514006C009EFB6
:10018A0011E0041B150BA80171E088279927443652
:10019A0018F4513008F404C0445650409395F7CFF0
:1001AA004A3018F04A508395FBCF02C099E089E0A3
:1001BA004427552708953330B0F410916500009113
:1001CA006400E016F10620F4F0926500E092640003
:1001DA0010916700009166000E151F0520F4F09239
:1001EA006700E0926600FF24EE24463D05E05007D2
:1001FA00C8F4443F01E0500710F44FEE51E04F5E5F
:10020A005140AA27BB27443618F4513008F404C0D9
:10021A0044565040B395F7CF4A3018F04A50A39548
:10022A00FBCF02C0A9E0B9E044275527089516B3C9
:10023A000C2F12FF0D2F0295007F08600BBB18953B
:10024A0000916900003019F00A9500936900109135
:10025A00680009B3087000936800101731F0109114
:10026A006900103011F403FF1DD013E003FF10934F
:10027A006900083029F010916A00139510936A00FA
:10028A0010916900103011F410936A0010916A00FD
:10029A00143629F411E010936A0003FF01C008958F
:1002AA0035D00895F8ECE395E53008F0E1E0E23066
:1002BA0079F0E330C1F0E430F9F0509161004091F7
:1002CA00600051DFEC0101E0070F046008BB0CCFAE
:1002DA00509163004091620046DFEC0101E0070F94
:1002EA00046008BB01CF50916500409164007DDF36
:1002FA00ED0104E008BBF8CE50916700409166001A
:10030A0074DFED0104E008BBEFCE0895FF27EE2766
:10031A00CC27DD2728E204E008BB0027009362000F
:10032A000093630000936600009367000FEF009349
:10033A0060000093640000936100009365000895D3
:00000001FF
